:0200000480007A
:100000006F00C004732F2034930F8000630AFF0336
:10001000930F90006306FF03930FB0006302FF038A
:10002000170F0080130F0FFE63040F0067000F000F
:10003000732F203463540F006F004000136E9E53E3
:10004000171F00002320CFFD6FF09FFF732540F1A5
:100050006310050073251030635805000F00F00F82
:10006000130E100073000000130E00009702000032
:10007000938282F973905230735020307350303035
:1000800073504030970200809382C2F7638C020065
:10009000739052109302B01A739022307323203061
:1000A000E39E62F873500030970200009382420191
:1000B00073901234732540F173002030B70001FFB4
:1000C000938000F037110F0F1301F1F0B3E120001E
:1000D000B70E10FF938EFEF0130E20006392D14BEB
:1000E000B710F00F938000FF37F1F0F01301010F0C
:1000F000B3E12000B70EF1FF938E0EFF130E300018
:100100006390D149B700FF009380F00F37110F0FB4
:100110001301F1F0B3E12000B71EFF0F938EFEFF35
:10012000130E4000639ED145B7F00FF09380F000AE
:1001300037F1F0F01301010FB3E12000B7FEFFF03B
:10014000938EFE0F130E5000639CD143B70001FF46
:10015000938000F037110F0F1301F1F0B3E020008E
:10016000B70E10FF938EFEF0130E6000639AD0411D
:10017000B70001FF938000F037110F0F1301F1F06A
:1001800033E12000B70E10FF938EFEF0130E7000C7
:100190006318D13FB70001FF938000F0B3E0100077
:1001A000B70E01FF938E0EF0130E8000639AD03DC0
:1001B00013020000B70001FF938000F037110F0F0A
:1001C0001301F1F0B3E120001383010013021200C8
:1001D00093022000E31052FEB70E10FF938EFEF044
:1001E000130E9000631ED33913020000B710F00FF6
:1001F000938000FF37F1F0F01301010FB3E120000D
:100200001300000013830100130212009302200068
:10021000E31E52FCB70EF1FF938E0EFF130EA000EB
:100220006310D33713020000B700FF009380F00F74
:1002300037110F0F1301F1F0B3E12000130000009C
:100240001300000013830100130212009302200028
:10025000E31C52FCB71EFF0F938EFEFF130EB0007F
:100260006310D33313020000B70001FF938000F046
:1002700037110F0F1301F1F0B3E120001302120048
:1002800093022000E31252FEB70E10FF938EFEF091
:10029000130EC0006396D12F13020000B710F00FA9
:1002A000938000FF37F1F0F01301010F13000000FD
:1002B000B3E120001302120093022000E31052FE6B
:1002C000B70EF1FF938E0EFF130ED000639AD12B61
:1002D00013020000B700FF009380F00F37110F0FDB
:1002E0001301F1F01300000013000000B3E120003F
:1002F0001302120093022000E31E52FCB71EFF0FF0
:10030000938EFEFF130EE000639CD12713020000C2
:10031000B70001FF938000F01300000037110F0FAA
:100320001301F1F0B3E12000130212009302200048
:10033000E31052FEB70E10FF938EFEF0130EF00086
:100340006390D12513020000B710F00F938000FFD7
:100350001300000037F1F0F01301010F130000004B
:10036000B3E120001302120093022000E31E52FCAE
:10037000B70EF1FF938E0EFF130E00016392D12191
:1003800013020000B700FF009380F00F130000007D
:100390001300000037110F0F1301F1F0B3E120003B
:1003A0001302120093022000E31E52FCB71EFF0F3F
:1003B000938EFEFF130E10016394D11D13020000F3
:1003C00037110F0F1301F1F0B70001FF938000F018
:1003D000B3E120001302120093022000E31252FE48
:1003E000B70E10FF938EFEF0130E2001639AD11901
:1003F0001302000037F1F0F01301010FB710F00FF6
:10040000938000FF13000000B3E1200013021200EC
:1004100093022000E31052FEB70EF1FF938E0EFF01
:10042000130E3001639ED1151302000037110F0F18
:100430001301F1F0B700FF009380F00F13000000EC
:1004400013000000B3E12000130212009302200009
:10045000E31E52FCB71EFF0F938EFEFF130E4001EA
:100460006390D1131302000037110F0F1301F1F045
:1004700013000000B70001FF938000F0B3E12000FB
:100480001302120093022000E31052FEB70E10FF79
:10049000938EFEF0130E50016394D10F13020000EF
:1004A00037F1F0F01301010F13000000B710F00F47
:1004B000938000FF13000000B3E12000130212003C
:1004C00093022000E31E52FCB70EF1FF938E0EFF45
:1004D000130E60016396D10B1302000037110F0F4A
:1004E0001301F1F01300000013000000B700FF003B
:1004F0009380F00FB3E1200013021200930220005A
:10050000E31E52FCB71EFF0F938EFEFF130E700109
:100510006398D107B70001FF938000F033611000AA
:10052000B70E01FF938E0EF0130E8001631AD105F2
:10053000B700FF009380F00F33E10000B70EFF001B
:10054000938EFE0F130E9001631CD103B360000065
:10055000930E0000130EA0016394D003B710111185
:1005600093801011372122221301212233E0200031
:10057000930E0000130EB0016314D001631CC00180
:100580000F00F00F63000E00131E1E00136E1E00FE
:10059000730000000F00F00F130E10007300000036
:1005A000731000C000000000000000000000000008
:1005B000000000000000000000000000000000003B
:0405C0000000000037
:1010000000000000000000000000000000000000E0
:1010100000000000000000000000000000000000D0
:1010200000000000000000000000000000000000C0
:1010300000000000000000000000000000000000B0
:081040000000000000000000A8
:040000058000200057
:00000001FF
